******************************************************************************
               TMS320C6x Linker PC v7.3.2                      
******************************************************************************
>> Linked Tue Feb 07 19:16:34 2012

OUTPUT FILE NAME:   <edmatset_C6678.out>
ENTRY POINT SYMBOL: "_c_int00"  address: 0c007f40


MEMORY CONFIGURATION

         name            origin    length      used     unused   attr    fill
----------------------  --------  ---------  --------  --------  ----  --------
  L1P                   00e00000   00007fff  00000000  00007fff  RWIX
  L1D                   00f00000   00007fff  00000000  00007fff  RWIX
  MSMC                  0c000000   001fffff  0000e0d0  001f1f2f  RWIX


SEGMENT ALLOCATION MAP

run origin  load origin   length   init length attrs members
----------  ----------- ---------- ----------- ----- -------
0c000000    0c000000    00008740   00008740    r-x
  0c000000    0c000000    00008740   00008740    r-x .text
0c008740    0c008740    00004000   00000000    rw-
  0c008740    0c008740    00002000   00000000    rw- .stack
  0c00a740    0c00a740    00002000   00000000    rw- .sysmem
0c00c740    0c00c740    00000a34   00000a34    r--
  0c00c740    0c00c740    00000a34   00000a34    r-- .const
0c00d180    0c00d180    00000a18   00000000    rw-
  0c00d180    0c00d180    00000a18   00000000    rw- .far
0c00dba0    0c00dba0    0000043c   0000031c    rw-
  0c00dba0    0c00dba0    0000031c   0000031c    rw- .fardata
  0c00debc    0c00debc    00000120   00000000    rw- .cio
0c00dfdc    0c00dfdc    00000108   00000108    r--
  0c00dfdc    0c00dfdc    00000070   00000070    r-- .switch
  0c00e04c    0c00e04c    00000098   00000098    r-- .cinit


SECTION ALLOCATION MAP

 output                                  attributes/
section   page    origin      length       input sections
--------  ----  ----------  ----------   ----------------
.text      0    0c000000    00008740     
                  0c000000    00001640     test.obj (.text)
                  0c001640    000005c0     rts6600_elf.lib : divd.obj (.text:__c6xabi_divd)
                  0c001c00    000005c0                     : _printfi.obj (.text:_getarg_diouxp)
                  0c0021c0    00000580     ti.csl.ae66 : csl_edma3HwChannelControl.oe66 (.text:csl_section:edma3:CSL_edma3HwChannelControl)
                  0c002740    00000520                 : csl_edma3HwControl.oe66 (.text:csl_section:edma3:CSL_edma3HwControl)
                  0c002c60    00000480     rts6600_elf.lib : _printfi.obj (.text:_setfield)
                  0c0030e0    00000460                     : _printfi.obj (.text:_printfi)
                  0c003540    00000300                     : fputs.obj (.text:fputs)
                  0c003840    000002e0                     : _printfi.obj (.text:_pproc_fwp)
                  0c003b20    000002e0     ti.csl.ae66 : csl_edma3GetHwStatus.oe66 (.text:csl_section:edma3:CSL_edma3GetHwStatus)
                  0c003e00    000002c0     rts6600_elf.lib : _printfi.obj (.text:_pproc_fge)
                  0c0040c0    000002a0                     : _printfi.obj (.text:fcvt)
                  0c004360    00000280                     : _printfi.obj (.text:ecvt)
                  0c0045e0    00000280                     : memory.obj (.text:free)
                  0c004860    00000240                     : imath64.obj (.text:__c6xabi_divull)
                  0c004aa0    00000240                     : _printfi.obj (.text:_pconv_e)
                  0c004ce0    00000240                     : _printfi.obj (.text:_pproc_diouxp)
                  0c004f20    00000220                     : _printfi.obj (.text:_pproc_str)
                  0c005140    00000200                     : _printfi.obj (.text:_pconv_g)
                  0c005340    000001c0                     : _printfi.obj (.text:_mcpy)
                  0c005500    000001c0                     : memory.obj (.text:malloc)
                  0c0056c0    000001a0                     : trgdrv.obj (.text:HOSTrename)
                  0c005860    000001a0                     : imath40.obj (.text:__c6xabi_divul)
                  0c005a00    00000180                     : copy_decompress_rle.obj (.text:__TI_decompress_rle_core)
                  0c005b80    00000180                     : autoinit.obj (.text:_auto_init_elf)
                  0c005d00    00000180                     : setvbuf.obj (.text:setvbuf)
                  0c005e80    00000140                     : _printfi.obj (.text:_pproc_fflags)
                  0c005fc0    00000140                     : fputc.obj (.text:fputc)
                  0c006100    00000140                     : lowlev.obj (.text:getdevice)
                  0c006240    00000120                     : _printfi.obj (.text:_ltostr)
                  0c006360    00000120                     : _io_perm.obj (.text:_wrt_ok)
                  0c006480    00000120     ti.csl.ae66 : csl_edma3ChannelOpen.oe66 (.text:csl_section:edma3:CSL_edma3ChannelOpen)
                  0c0065a0    00000120                 : csl_edma3GetBaseAddress.oe66 (.text:csl_section:edma:CSL_edma3ccGetModuleBaseAddr)
                  0c0066c0    00000120     rts6600_elf.lib : fclose.obj (.text:fclose)
                  0c0067e0    00000100                     : trgdrv.obj (.text:HOSTlseek)
                  0c0068e0    00000100                     : cpy_tbl.obj (.text:copy_in)
                  0c0069e0    000000e0                     : trgdrv.obj (.text:HOSTopen)
                  0c006ac0    000000e0                     : _printfi.obj (.text:_div)
                  0c006ba0    000000e0                     : atoi.obj (.text:atoi)
                  0c006c80    000000e0                     : lowlev.obj (.text:close)
                  0c006d60    000000e0                     : copy_zero_init.obj (.text:decompress:ZI:__TI_zero_init)
                  0c006e40    000000e0                     : exit.obj (.text:exit)
                  0c006f20    000000e0                     : ltoa.obj (.text:ltoa)
                  0c007000    000000e0                     : memset.obj (.text:memset)
                  0c0070e0    000000c0                     : trgdrv.obj (.text:HOSTread)
                  0c0071a0    000000c0                     : trgdrv.obj (.text:HOSTunlink)
                  0c007260    000000c0                     : trgdrv.obj (.text:HOSTwrite)
                  0c007320    000000c0                     : divu.obj (.text:__divu)
                  0c0073e0    000000c0                     : fopen.obj (.text:_cleanup)
                  0c0074a0    000000c0                     : fflush.obj (.text:_doflush)
                  0c007560    000000c0     ti.csl.ae66 : csl_edma3HwChannelSetup.oe66 (.text:csl_section:edma3:CSL_edma3HwChannelSetupQue)
                  0c007620    000000c0                 : csl_edma3Open.oe66 (.text:csl_section:edma3:CSL_edma3Open)
                  0c0076e0    000000c0     rts6600_elf.lib : fseek.obj (.text:fseek)
                  0c0077a0    000000c0                     : lowlev.obj (.text:lseek)
                  0c007860    000000c0                     : lowlev.obj (.text:write)
                  0c007920    000000a0                     : trgdrv.obj (.text:HOSTclose)
                  0c0079c0    000000a0                     : _printfi.obj (.text:_ecpy)
                  0c007a60    000000a0                     : _printfi.obj (.text:_fcpy)
                  0c007b00    000000a0                     : _printfi.obj (.text:_pconv_f)
                  0c007ba0    000000a0     ti.csl.ae66 : csl_edma3HwChannelSetup.oe66 (.text:csl_section:edma3:CSL_edma3HwChannelSetupParam)
                  0c007c40    000000a0     rts6600_elf.lib : lowlev.obj (.text:finddevice)
                  0c007ce0    000000a0                     : memcpy64.obj (.text:memcpy)
                  0c007d80    000000a0                     : memory.obj (.text:minsert)
                  0c007e20    000000a0                     : memory.obj (.text:mremove)
                  0c007ec0    00000080                     : llshift.obj (.text:__c6xabi_llshl)
                  0c007f40    00000080                     : boot.obj (.text:_c_int00)
                  0c007fc0    00000080                     : memory.obj (.text:_minit)
                  0c008040    00000080     ti.csl.ae66 : csl_edma3Param.oe66 (.text:csl_section:edma3:CSL_edma3GetParamHandle)
                  0c0080c0    00000080                 : csl_edma3HwChannelSetup.oe66 (.text:csl_section:edma3:CSL_edma3HwChannelSetupTriggerWord)
                  0c008140    00000080     rts6600_elf.lib : printf.obj (.text:printf)
                  0c0081c0    00000080                     : trgmsg.obj (.text:readmsg)
                  0c008240    00000080                     : lowlev.obj (.text:unlink)
                  0c0082c0    00000060                     : frcmpyd_div.obj (.text:__c6xabi_frcmpyd_div)
                  0c008320    00000060                     : llshift.obj (.text:__c6xabi_llshru)
                  0c008380    00000060                     : imath64.obj (.text:_subcull)
                  0c0083e0    00000060     ti.csl.ae66 : csl_edma3Param.oe66 (.text:csl_section:edma3:CSL_edma3ParamSetup)
                  0c008440    00000060     rts6600_elf.lib : memccpy.obj (.text:memccpy)
                  0c0084a0    00000060                     : trgmsg.obj (.text:writemsg)
                  0c008500    00000040                     : isinf.obj (.text:__c6xabi_isinf)
                  0c008540    00000040                     : _printfi.obj (.text:__c6xabi_isnan)
                  0c008580    00000040                     : args_main.obj (.text:_args_main)
                  0c0085c0    00000040     ti.csl.ae66 : csl_edma3ChannelClose.oe66 (.text:csl_section:edma3:CSL_edma3ChannelClose)
                  0c008600    00000020     rts6600_elf.lib : negll.obj (.text:__c6xabi_negll)
                  0c008620    00000020                     : _lock.obj (.text:_nop)
                  0c008640    00000020                     : printf.obj (.text:_outc)
                  0c008660    00000020                     : printf.obj (.text:_outs)
                  0c008680    00000020                     : exit.obj (.text:abort)
                  0c0086a0    00000020     ti.csl.ae66 : csl_edma3Close.oe66 (.text:csl_section:edma3:CSL_edma3Close)
                  0c0086c0    00000020                 : csl_edma3Init.oe66 (.text:csl_section:edma3:CSL_edma3Init)
                  0c0086e0    00000020                 : csl_edma3Param.oe66 (.text:csl_section:edma3:CSL_edma3ParamWriteWord)
                  0c008700    00000020     rts6600_elf.lib : copy_decompress_none.obj (.text:decompress:none:__TI_decompress_none)
                  0c008720    00000020                     : copy_decompress_rle.obj (.text:decompress:rle24:__TI_decompress_rle24)

.stack     0    0c008740    00002000     UNINITIALIZED
                  0c008740    00000008     rts6600_elf.lib : boot.obj (.stack)
                  0c008748    00001ff8     --HOLE--

.sysmem    0    0c00a740    00002000     UNINITIALIZED
                  0c00a740    00000008     rts6600_elf.lib : memory.obj (.sysmem)
                  0c00a748    00001ff8     --HOLE--

.const     0    0c00c740    00000a34     
                  0c00c740    0000090c     test.obj (.const:.string)
                  0c00d04c    00000004     --HOLE-- [fill = 0]
                  0c00d050    00000101     rts6600_elf.lib : ctype.obj (.const:_ctypes_)
                  0c00d151    00000023                     : _printfi.obj (.const:.string)

.far       0    0c00d180    00000a18     UNINITIALIZED
                  0c00d180    00000800     test.obj (.far)
                  0c00d980    00000140     rts6600_elf.lib : defs.obj (.far)
                  0c00dac0    000000d8                     : trgdrv.obj (.far)

.fardata   0    0c00dba0    0000031c     
                  0c00dba0    000001e0     rts6600_elf.lib : defs.obj (.fardata:_ftable)
                  0c00dd80    000000a0                     : lowlev.obj (.fardata:_stream)
                  0c00de20    00000078                     : lowlev.obj (.fardata:_device)
                  0c00de98    0000000c                     : exit.obj (.fardata)
                  0c00dea4    0000000c                     : memory.obj (.fardata)
                  0c00deb0    00000008                     : _lock.obj (.fardata)
                  0c00deb8    00000004                     : defs.obj (.fardata)

.cio       0    0c00debc    00000120     UNINITIALIZED
                  0c00debc    00000120     rts6600_elf.lib : trgmsg.obj (.cio)

.switch    0    0c00dfdc    00000070     
                  0c00dfdc    0000003c     ti.csl.ae66 : csl_edma3HwControl.oe66 (.switch:CSL_edma3HwControl)
                  0c00e018    00000020                 : csl_edma3GetHwStatus.oe66 (.switch:CSL_edma3GetHwStatus)
                  0c00e038    00000014                 : csl_edma3HwChannelControl.oe66 (.switch:CSL_edma3HwChannelControl)

.cinit     0    0c00e04c    00000098     
                  0c00e04c    00000072     (.cinit..fardata.load) [load image, compression = rle]
                  0c00e0be    00000002     --HOLE-- [fill = 0]
                  0c00e0c0    0000000c     (__TI_handler_table)
                  0c00e0cc    00000008     (.cinit..far.load) [load image, compression = zero_init]
                  0c00e0d4    00000010     (__TI_cinit_table)


LINKER GENERATED COPY TABLES

__TI_cinit_table @ 0c00e0d4 records: 2, size/record: 8, table size: 16
	.fardata: load addr=0c00e04c, load size=00000072 bytes, run addr=0c00dba0, run size=0000031c bytes, compression=rle
	.far: load addr=0c00e0cc, load size=00000008 bytes, run addr=0c00d180, run size=00000a18 bytes, compression=zero_init


LINKER GENERATED HANDLER TABLE

__TI_handler_table @ 0c00e0c0 records: 3, size/record: 4, table size: 12
	index: 0, handler: __TI_zero_init
	index: 1, handler: __TI_decompress_rle24
	index: 2, handler: __TI_decompress_none


GLOBAL SYMBOLS: SORTED ALPHABETICALLY BY Name 

address    name
--------   ----
0c008680   C$$EXIT
0c0084f8   C$$IO$$
0c0085c0   CSL_edma3ChannelClose
0c006480   CSL_edma3ChannelOpen
0c0086a0   CSL_edma3Close
0c003b20   CSL_edma3GetHwStatus
0c008040   CSL_edma3GetParamHandle
0c0021c0   CSL_edma3HwChannelControl
0c007ba0   CSL_edma3HwChannelSetupParam
0c007560   CSL_edma3HwChannelSetupQue
0c0080c0   CSL_edma3HwChannelSetupTriggerWord
0c002740   CSL_edma3HwControl
0c0086c0   CSL_edma3Init
0c007620   CSL_edma3Open
0c0083e0   CSL_edma3ParamSetup
0c0086e0   CSL_edma3ParamWriteWord
0c0065a0   CSL_edma3ccGetModuleBaseAddr
0c007920   HOSTclose
0c0067e0   HOSTlseek
0c0069e0   HOSTopen
0c0070e0   HOSTread
0c0056c0   HOSTrename
0c0071a0   HOSTunlink
0c007260   HOSTwrite
0c00debc   __CIOBUF_
0c00e0d4   __TI_CINIT_Base
0c00e0e4   __TI_CINIT_Limit
0c00e0c0   __TI_Handler_Table_Base
0c00e0cc   __TI_Handler_Table_Limit
0c00a740   __TI_STACK_END
00002000   __TI_STACK_SIZE
00000000   __TI_STATIC_BASE
00002000   __TI_SYSMEM_SIZE
00000001   __TI_args_main
0c008700   __TI_decompress_none
0c008720   __TI_decompress_rle24
0c00dea0   __TI_enable_exit_profile_output
ffffffff   __TI_pprof_out_hndl
ffffffff   __TI_prof_data_size
ffffffff   __TI_prof_data_start
0c006d60   __TI_zero_init
ffffffff   __binit__
0c001640   __c6xabi_divd
0c007320   __c6xabi_divu
0c005860   __c6xabi_divul
0c004860   __c6xabi_divull
0c0082c0   __c6xabi_frcmpyd_div
0c008500   __c6xabi_isinf
0c007ec0   __c6xabi_llshl
0c008320   __c6xabi_llshru
0c008600   __c6xabi_negll
ffffffff   __c_args__
0c007320   __divu
0c008580   _args_main
0c005b80   _auto_init_elf
0c007f40   _c_int00
0c0073e0   _cleanup
0c00de98   _cleanup_ptr
0c00d050   _ctypes_
0c0074a0   _doflush
0c00de9c   _dtors_ptr
0c00deb8   _ft_end
0c00dba0   _ftable
0c00deb0   _lock
0c007fc0   _minit
0c008620   _nop
0c0030e0   _printfi
0c008740   _stack
0c008380   _subcull
0c00a740   _sys_memory
0c00d980   _tmpnams
0c00deb4   _unlock
0c006360   _wrt_ok
0c008680   abort
0c006ba0   atoi
ffffffff   binit
0c006c80   close
0c0068e0   copy_in
0c00d580   dstBuff1
0c00d780   dstBuff2
0c006e40   exit
0c0066c0   fclose
0c005fc0   fputc
0c003540   fputs
0c0045e0   free
0c0076e0   fseek
0c0077a0   lseek
0c006f20   ltoa
0c001180   main
0c005500   malloc
0c008440   memccpy
0c007ce0   memcpy
0c007000   memset
0c008140   printf
0c005fc0   putc
0c0081c0   readmsg
0c008240   remove
0c005d00   setvbuf
0c00d180   srcBuff1
0c00d380   srcBuff2
0c008240   unlink
0c007860   write
0c0084a0   writemsg


GLOBAL SYMBOLS: SORTED BY Symbol Address 

address    name
--------   ----
00000000   __TI_STATIC_BASE
00000001   __TI_args_main
00002000   __TI_STACK_SIZE
00002000   __TI_SYSMEM_SIZE
0c001180   main
0c001640   __c6xabi_divd
0c0021c0   CSL_edma3HwChannelControl
0c002740   CSL_edma3HwControl
0c0030e0   _printfi
0c003540   fputs
0c003b20   CSL_edma3GetHwStatus
0c0045e0   free
0c004860   __c6xabi_divull
0c005500   malloc
0c0056c0   HOSTrename
0c005860   __c6xabi_divul
0c005b80   _auto_init_elf
0c005d00   setvbuf
0c005fc0   fputc
0c005fc0   putc
0c006360   _wrt_ok
0c006480   CSL_edma3ChannelOpen
0c0065a0   CSL_edma3ccGetModuleBaseAddr
0c0066c0   fclose
0c0067e0   HOSTlseek
0c0068e0   copy_in
0c0069e0   HOSTopen
0c006ba0   atoi
0c006c80   close
0c006d60   __TI_zero_init
0c006e40   exit
0c006f20   ltoa
0c007000   memset
0c0070e0   HOSTread
0c0071a0   HOSTunlink
0c007260   HOSTwrite
0c007320   __c6xabi_divu
0c007320   __divu
0c0073e0   _cleanup
0c0074a0   _doflush
0c007560   CSL_edma3HwChannelSetupQue
0c007620   CSL_edma3Open
0c0076e0   fseek
0c0077a0   lseek
0c007860   write
0c007920   HOSTclose
0c007ba0   CSL_edma3HwChannelSetupParam
0c007ce0   memcpy
0c007ec0   __c6xabi_llshl
0c007f40   _c_int00
0c007fc0   _minit
0c008040   CSL_edma3GetParamHandle
0c0080c0   CSL_edma3HwChannelSetupTriggerWord
0c008140   printf
0c0081c0   readmsg
0c008240   remove
0c008240   unlink
0c0082c0   __c6xabi_frcmpyd_div
0c008320   __c6xabi_llshru
0c008380   _subcull
0c0083e0   CSL_edma3ParamSetup
0c008440   memccpy
0c0084a0   writemsg
0c0084f8   C$$IO$$
0c008500   __c6xabi_isinf
0c008580   _args_main
0c0085c0   CSL_edma3ChannelClose
0c008600   __c6xabi_negll
0c008620   _nop
0c008680   C$$EXIT
0c008680   abort
0c0086a0   CSL_edma3Close
0c0086c0   CSL_edma3Init
0c0086e0   CSL_edma3ParamWriteWord
0c008700   __TI_decompress_none
0c008720   __TI_decompress_rle24
0c008740   _stack
0c00a740   __TI_STACK_END
0c00a740   _sys_memory
0c00d050   _ctypes_
0c00d180   srcBuff1
0c00d380   srcBuff2
0c00d580   dstBuff1
0c00d780   dstBuff2
0c00d980   _tmpnams
0c00dba0   _ftable
0c00de98   _cleanup_ptr
0c00de9c   _dtors_ptr
0c00dea0   __TI_enable_exit_profile_output
0c00deb0   _lock
0c00deb4   _unlock
0c00deb8   _ft_end
0c00debc   __CIOBUF_
0c00e0c0   __TI_Handler_Table_Base
0c00e0cc   __TI_Handler_Table_Limit
0c00e0d4   __TI_CINIT_Base
0c00e0e4   __TI_CINIT_Limit
ffffffff   __TI_pprof_out_hndl
ffffffff   __TI_prof_data_size
ffffffff   __TI_prof_data_start
ffffffff   __binit__
ffffffff   __c_args__
ffffffff   binit

[103 symbols]
